:020000040000FA
:040000000CD0EFD061
:08000800FFD082BEF4D0040019
:0600100082AEFED71200D3
:08001800FFD0A66AA968AA68DE
:10002000A680A84A05D0A84CEBD0066E310ECD6E46
:10003000800E946E900EAB6E260EAC6EAB98030ED7
:10004000D56ED76AD66AD7D8D58ED5D8D59ED6CF15
:1000500003F0D7320332D8A0030603C0AFFFAB884A
:10006000AE50AE50B6D80F0AE9E100EE08F0006AD3
:10007000016AAFD80F0AF6E00450040A0AE00450FF
:10008000050A01E1A6D804500026EE6E014ED6D72F
:10009000F0D70052D3E1CD900A50F66EA96E0B5006
:1000A000F76EAA6E0CC0F8FF00EE0DF00950016E5D
:1000B000D8B4FF0008500808C1E3FA6AFB6A084494
:1000C000F92608D01ED025D034D03ED048D019D043
:1000D00052D0FF00EE50AF02F446F446FC0EF41688
:1000E000F346F346030EF314F424A86E040EA66E32
:1000F00078D8A6B2FED70C0E0A6E000E0B6E040E58
:1001000045D00900F5CFEEFF012EFBD70950050FB2
:100110003DD0F80EF616080EEECFF5FF0D00E82ED6
:10012000FBD70A00840EA66E5CD80900012EF1D719
:100130002CD0940EA66E55D8400EF626E86AF7220B
:10014000F822012EF6D721D0A66AA680A8CFEEFF0E
:10015000A94AAA2A012EF8D70950050F17D0EECFC9
:10016000A8FF040EA66E3DD8A6B2FED7A94AAA2AB9
:10017000012EF5D70AD0C40EA66EEECFF5FF0C0007
:1001800030D80900012EF7D700D0010E016E0F0EF6
:100190001BD81AD8006A00EE08F0EE50002608D8E6
:1001A000012EFBD7006C005003D8040E0DD846D7A3
:1001B000056E0F0A06E00550040A03E00550050A23
:1001C00002E1050E01D8055004009EA8FED7AD6ED1
:1001D00012000400ABB2FF009EAAFED7AE50046E20
:1001E00012000400550EA76EAA0EA76EA68200008C
:0201F0001200FB
:0A01F6009EA008D79E90062E05D7A4
:020000040030CA
:0E000000FFFAFCFEFFFFFBFFFFFFFFFFFFFF0D
:00000001FF
